:020000040000FA
:10000000543083169000831207309900FF3085002A
:1000100083167F30810000309500183085008312F0
:10002000FF3085000030A5000730A40019307D2086
:1000300004307D200510822005147C2025185428CA
:100040008510822085147C202518542805118220D3
:1000500005157C20251854288512822085167C20C1
:100060002518542883160830850083120512412074
:10007000051683161830850083127C202518542815
:100080001A280430A200FA30A1006F30A00000004E
:1000900000000000000000000000A00B4728A10B9A
:1000A0004528A20B432800348316FF3085008312B5
:1000B0006B20051E5E280000000059286B200030D0
:1000C000A50000000000051E612883161830850079
:1000D000831282201A28FA30A1006F30A00000009D
:1000E00000000000000000000000A00B6F28A10B22
:1000F0006D28051E6B2800342408A3008220A30B62
:100100007E2800340430A200FA30A1006F30A00035
:10011000051E972825189728000000000000000001
:10012000A00B8828A10B8628A20B8428003401305C
:10013000A500A000A100A200A3008C282A00450071
:100140006D0069006C0069006F002A002800310012
:1001500039002D00300035002D0030003700290017
:040160000034003433
:02400E00843FED
:00000001FF
